:100000000C94ED020C9434030C9434030C943403DC
:100010000C9434030C9434030C9434030C94340384
:100020000C9434030C9434030C94EE240C94C225E9
:100030000C944D1F0C9434030C9434030C9434032F
:100040000C9434030C9434030C9434030C94340354
:100050000C9434030C94A41F0C9434030C943403B8
:100060000C9434030C9434030C9434030C94340334
:100070000C9434030C9434030C9434030C94340324
:100080000C9434030C9434030C9434030C94340314
:100090000C9434030C9434030C9434030C94340304
:1000A0000C9434030C9434030C94340300000000CB
:1000B0000000000000000000000000000000000040
:1000C0000000000000000000000000000000000030
:1000D0000000000000061E3EFEFEFCFCFCFCFCFCDA
:1000E000FCFCFCFCFCFCFCFCFCFCFCFCFCFCFCFC50
:1000F000FCFCFCFCFCFCFCFCFCFCFCFCFCFEFE3EFA
:100100001E060000000000000000000000000000CB
:1001100000000000000000000000000000000000DF
:1001200000000000000000000000000000000000CF
:1001300000000000000000000000000000000000BF
:1001400000000000000000000000000000000000AF
:100150000002060E1E3E3EFEFEFF7F7FFFFF7F7FFA
:100160007F7F7F7F0F0F0F0F0F0F0F0F0F0F0F0FDF
:100170000F0F0F7F7F7F7F7FFFFFFF7F7FFFFEFEE1
:100180003E3E1E0E060200000000000000000000BF
:10019000000000000000000000000000000000005F
:1001A000000000000000000000000000000000004F
:1001B000000000000000000000000000000000003F
:1001C000000000000000000000000000000000002F
:1001D0000000000000E0FCFF070000F8FF1F000027
:1001E000000000000000000000000000000000000F
:1001F0000000000000000000001FFFF800000FFFDB
:10020000FEE0000000000000000000000000000010
:1002100000000000000000000000000000000000DE
:1002200000000000000000000000000000000000CE
:1002300000000000000000000000000000000000BE
:1002400000000000000000000000000000000000AE
:10025000000000383F3F0F0000001F1F0F0000008C
:10026000000000000000000000000000000000008E
:1002700000000000000000000000071F1F00000039
:10028000073F3F30000000000000000000000000B9
:10029000000000000000000000000000000000005E
:1002A000000000000000000000000000AC00AE00F4
:1002B000AB00AD00AF00A8003A003B003C003D00A1
:1002C0003E004B0000007C0000007D0000004E005E
:1002D0000100010001000100010001000100010016
:1002E0000100010001000100010001000000010007
:1002F00000000100010001000100010001000100F7
:1003000001000100010001000100010001000100E5
:1003100000000100000001000100010001000100D7
:1003200001000100010001000100010001000100C5
:1003300001000100000001000000010000000000B9
:10034000000000002A2B2800000000000000000030
:100350000000000000000029000000002C1E3420D6
:10036000212224342627252E362D3738271E1F20FC
:100370002122232425263333362E37381F04050641
:100380000708090A0B0C0D0E0F1011121314151685
:100390001718191A1B1C1D2F3130232D3504050683
:1003A0000708090A0B0C0D0E0F1011121314151665
:1003B0001718191A1B1C1D2F3130354C0000000076
:1003C000000000000000000000000000000000002D
:1003D000000000000000000000000000000000001D
:1003E0007E0F00D4FFFFFFC70000007800AE00AF13
:1003F00000DA0281FFD9F1DB20A4A62EAF00A0C055
:1004000000A1C800AED580A81FD300408D142000E5
:100410001003440061006D00610070006100640021
:1004200000002C0342006F006C007300610020008C
:100430004B006500790062006F006100720064008B
:10044000200053007500700070006C0079000000FF
:100450000403090409025B00030100A0FA09040077
:1004600000010301010009211101000122400007E0
:1004700005810308000A09040100020300000009C5
:10048000211101000122220007058203200001073B
:100490000503032000010904020001030000000914
:1004A000211101000122B6000705840320000A1271
:1004B00001000200000008646D7064010001020088
:1004C000010660FF0961A1010962150026FF009580
:1004D00020750881020963150026FF009520750824
:1004E0009102C005010902A10185020901A10005CF
:1004F00009190129081500250195087501810205D2
:1005000001093009311581257F9502750881060999
:10051000381581257F950175088106050C0A38027A
:100520001581257F950175088106C0C005010980E8
:10053000A101850319012AB700150126B70095010D
:1005400075108100C0050C0901A101850419012A5B
:10055000A002150126A002950175108100C00501B9
:100560000906A1018506050719E029E715002501FF
:100570009508750181020507190029EF150025016D
:1005800095F0750181020508190129059505750188
:100590009102950175039101C005010906A10105AC
:1005A0000719E029E71500250195087501810295D5
:1005B00001750881010507190029FF150026FF00B4
:1005C000950675088100050819012905950575012D
:1005D0009102950175039101C00011241FBECFEF58
:1005E000DAE0DEBFCDBF04B603FE27C08091B804B9
:1005F0009091B904A091BA04B091BB048730904B9C
:10060000A740B04BD1F41092B8041092B9041092E4
:10061000BA041092BB0414BE84B7877F84BF0FB6A0
:10062000F894A89580916000886180936000109292
:1006300060000FBEE0E0F8E3099511E0A0E0B1E052
:10064000E2E6F0E502C005900D92A23BB107D9F7B2
:1006500024E0A2EBB1E001C01D92A83BB207E1F794
:100660000E9498120C94F8270C94000060E072E04D
:100670008CEA90E00E94141780E0089582E00895CB
:10068000662339F06AE070E089EA0E94E90580E0BB
:1006900008956AE070E08AEAF8CF81E0089581E089
:1006A00008950C944F0308950C9453031F93CF9314
:1006B000DF9300D000D00F92CDB7DEB749835A83C5
:1006C0006B833091B40189819A8131111DC06623F9
:1006D000B9F02223A9F00E947209182F682F89818E
:1006E0009A810E941B0969817A81812F0F900F9056
:1006F0000F900F900F90DF91CF911F910C94A91A3A
:100700000E944909182FEFCF0E94720969817A81EE
:10071000EDCFFC01262F408151816281738184815C
:100720000C94560381E00895CF93DF93EC0160E0D1
:100730000E948903BE01DF91CF910C945403E1E044
:10074000F0E0DF0102C0AA0FBB1F6A95E2F7BD010E
:10075000DF0102C0AA0FBB1F4A95E2F76A2B01C056
:10076000EE0F2A95EAF7962F9823961302C08E2B48
:100770000895E0958E230895242F462F682F8091A9
:10078000BE010E949F030C94D8080E9439110E9458
:1007900020050C9454110C945711089508950C944D
:1007A000CE030E94CF0380E00E9421050C947018B4
:1007B00008950E9470080E94D8032FEF84E39CE004
:1007C000215080409040E1F700C000000C94C81F09
:1007D0000F931F93CF93DF938C0161E00E948903F5
:1007E000EC01B8010E9487158823D9F1B801CE0128
:1007F0000E9451038823A9F1B801CE010E946E1C0A
:10080000882379F1B801CE010E94B918882349F1F3
:10081000B801CE010E94D81B882319F1F80182810A
:10082000882361F0CA35FDE5DF0721F170F4C115B9
:10083000ECE5DE07A1F0CE3DDC45C9F0C801DF9153
:10084000CF911F910F910C944D03CB358DE5D807B7
:10085000A1F0CC35DD4591F70E94850DEFCF0E94C8
:10086000D90380E0DF91CF911F910F9108950E94ED
:100870003E0EF7CF0E948E0DE1CF0E94910DDECF8C
:100880000C94CD030E94D11D0E9421050C944004BC
:10089000DF92EF92FF920F931F93CF93DF93E82F96
:1008A000F0E0E45CFC4FD490282F26952695269501
:1008B00030E0F901E452FC4F0491877010E0082EFB
:1008C00002C0159507950A94E2F701701127F90106
:1008D000E453FC4FE490F12C082E02C0F594E79409
:1008E0000A94E2F791E0E922FF24F901E454FC4F75
:1008F000C491D0E002C0D595C7958A95E2F7C17042
:10090000DD270115110519F081EE0E946C05E11437
:10091000F10419F086EE0E946C058D2D0E940006F0
:10092000EF2819F086EE0E94BA05012B19F081EE2E
:100930000E94BA05CD2B51F08CE2DF91CF911F912F
:100940000F91FF90EF90DF900C940006DF91CF9114
:100950001F910F91FF90EF90DF900895EF92FF921B
:100960000F931F93CF93DF93EC01162F0AE088813A
:10097000882309F454C0813009F04EC08981813048
:1009800099F47E0122E0E20EF11C8A810E940006A9
:10099000E7012196812F815050F3EFE9FFE0319775
:1009A000F1F700C00000F7CF823041F47E0182E011
:1009B000E80EF11C8A810E946C05EACF833041F475
:1009C0007E01E2E0EE0EF11C8A810E94BA05E0CFC2
:1009D000843011F02196DDCF2A81229690E080E0CC
:1009E000AE014F5F5F4F2053330B2A30310548F083
:1009F000019778F2EFE9FFE03197F1F700C00000CE
:100A0000F7CF089FB001099F700D1124C901860F0F
:100A1000971F2981EA01E4CF0E944804BACFDF91F1
:100A2000CF911F910F91FF90EF90089560E00C948B
:100A3000AE0408950C94190581E008950C941C05EA
:100A40000895CF93C82F0E941A058C2FCF910C9434
:100A50001E05CF93DF93CDB7DEB72B970FB6F89473
:100A6000DEBF0FBECDBF4F83588769877A878B87DC
:100A700061110E94E00C1E821D8285E0FE01379606
:100A8000DE01119601900D928A95E1F78C819D818E
:100A9000892B89F449815A816B817C818D819E816A
:100AA0000E94010C2B960FB6F894DEBF0FBECDBF8F
:100AB000DF91CF91089589819A8189238F3F51F3E6
:100AC000CE0101960E9492038111E4CFEBCFFC018D
:100AD000808191810C949F09CF93C82F882309F4BA
:100AE00047C08CEF8C0F813AA0F46C2F80910201EB
:100AF000909103010E94451E882329F08C2F0E94AB
:100B0000A20C0E94030D8C2F0E949B0CCF910C9481
:100B1000030D80E28C0F883048F4C77081E001C07B
:100B2000880FCA95EAF70E94C30CF0CFEBE5EC0FF3
:100B3000E33040F4F0E0E25BFE4F808190E0CF9143
:100B40000C94051EE8E5EC0FE73150F4F0E0EE0FF1
:100B5000FF1FE05EFE4F80819181CF910C941B1EA0
:100B6000C03F30F08C2F0E942813CF910C94FB13C0
:100B7000CF910895882361F19CEF980F913A20F46A
:100B80000E94A20C0C94030D90E2980F983050F440
:100B9000877091E001C0990F8A95EAF7892F0E942A
:100BA000C90CF0CF9BE5980F933020F490E080E0E3
:100BB0000C94051E98E5980F973120F490E080E0A2
:100BC0000C941B1E803F20F00E9482130C94FB1398
:100BD00008951F93CF93DF93182FEB010E946C05AC
:100BE000209731F4812FDF91CF911F910C94BA059A
:100BF0008FE99FE00197F1F700C000002197F0CF47
:100C000070E060E0893311F460E570E00C94E90570
:100C1000882321F00E94C30C0C94030D08958823AF
:100C200021F00E94C90C0C94030D0895BF92CF923D
:100C3000DF92EF92FF920F931F93CF93DF936C019C
:100C4000D62FC72FFC011281F580F2949FE0F92284
:100C50000E94B90CE82E8823B9F0E12E1123A1F0EF
:100C60008C2F807F803421F080E28D0F8830D0F08F
:100C700080919A0282FD16C082E00E94540D0E946B
:100C8000B90C91E0E82EE926BC2EB2948FE0B82290
:100C9000FBE0FB1508F468C0EB2DF0E0E650F84DE2
:100CA0000C949C27E12CF0CF0C2F0F70C07F11F01B
:100CB0000295007F112399F0002359F080E28D0FF7
:100CC000883010F0D11107C0802F0E94C30C0E9401
:100CD000030D8D2F41C0802F0E94D30CF8CF8D2F94
:100CE0000E94BA05002309F43FC080E28D0F8830CE
:100CF00010F0D11104C0802F0E94C90C03C0802FB6
:100D00000E94D90C0E94030D2FC00C2F0F70C07FC2
:100D1000C03211F00295007FDD2381F0D13009F45B
:100D200069C0112309F473C0FF2009F469C0F601FA
:100D3000858180FFCECF8F70858362C080919A02BB
:100D400082FF38C0112359F0002329F0802F0E9420
:100D5000C30C0E94030D80E00E946C0505C080E07A
:100D60000E94BA050111C7CFEB2DE850FF0B349755
:100D700020F40E94D11D0E942105EE2009F44DC1EE
:100D80000E94B50C80FD49C1F60112820E94AF0C91
:100D90000E94E908C6010E942E080E94AF0CDF9154
:100DA000CF911F910F91FF90EF90DF90CF90BF9068
:100DB0000C94F408112389F0F11006C00E94E60C8F
:100DC000802B0E940806D0CF21E0F212F7CF0E94BC
:100DD000E60C802B0E94EC0CC7CFF11006C00E94DD
:100DE000F90C802F0E940F06BFCF31E0F31609F4F3
:100DF000BBCFF5CF112331F085E08F1508F4B4CFC8
:100E0000802FDFCF94E09F1508F4AECFEACFFF200C
:100E100041F3D93349F4FFEF27EE33E0F15020409E
:100E20003040E1F700C000008D2F0E94BA059CCF32
:100E30008C2F86958695837069F0813009F094CF68
:100E40008D2F9C2F9370111102C090E080E00E94C2
:100E50001B1E8ACF8D2F9C2F9370111102C090E022
:100E600080E00E94051E80CF8D2F112329F00E9463
:100E700028130E94FB1378CF0E948213FACF8C2F85
:100E8000837079F5111170CF4D2F429546954770BB
:100E9000440F440F8D2F8F70042E01C0880F0A94C9
:100EA000EAF72D2F2071D4FF07C02FE030E001C0FA
:100EB000220F4A95EAF72095C695C695C370822BF6
:100EC000C23049F058F4C13019F00E94CA084CCF22
:100ED0000E94C50849CF0E94CF0846CF0E94C30890
:100EE00043CF8695112311F08C2F8170882309F44C
:100EF0003BCF4D2F429546954770440F440F8D2FA1
:100F00008F70042E01C0880F0A94EAF72D2F2071EC
:100F1000D4FF07C02FE030E001C0220F4A95EAF766
:100F20002095C695C695C370822BC23049F058F4FF
:100F3000C13019F00E94100917CF0E940B0914CF7D
:100F40000E94150911CF0E94D8080ECFCF7011232F
:100F500029F08C2F0E94E9088D2F33CF8D2F0E940E
:100F60000F068C2F0E94F408FFCED23F51F160F49F
:100F7000D03FB9F0D13F81F0112309F449C0F110FD
:100F8000A8CE8C2F8F7121C0D33F11F1D43FA1F790
:100F900080919A0282FF26C08C2F8F71112311F34A
:100FA00014C0112349F084E08F1508F4DDCE8C2F96
:100FB0008F710E940009D8CE95E09F1508F4D4CE19
:100FC000F6CF8C2F8F711111CDCF0E94E908CCCEB6
:100FD000112329F08C2F8F710E94E108C5CE0E9449
:100FE000DE08C2CE112349F0CF718C2F0E94E90890
:100FF00063E08C2F0E94390DB7CE81E00E94540D22
:10100000E1E0EF1508F0B0CE82E00E94540DACCEC6
:10101000F110FFCE8C2F8F71A5CFDF91CF911F9153
:101020000F91FF90EF90DF90CF90BF9008950F93B6
:101030001F93CF93DF93EC01688179818A810E94AD
:10104000A9098C010E941A090E94C208B801CE01A8
:10105000DF91CF911F910F910C941606CF93DF93E0
:10106000EC018B819C81892B29F0888199818923CE
:101070008F3F59F4DF91CF910895CE010E94170858
:10108000CE01DF91CF910C949403CE010E94E8032E
:101090008111F3CF0E94B90C882361F38A818823E0
:1010A00049F380919A0282FDE5CF82E0DF91CF91F2
:1010B0000C94540D90E080E00E94051E90E080E0CA
:1010C0000E941B1E0E94E00C0E94E30C0E94030D74
:1010D0000E9422150C94FB130E94A90C0C945A0830
:1010E0000E94D00C0C946C08E92FE295EF70E2504E
:1010F000EE3070F4F0E0EA5FF74D0C949C27803FEF
:1011000019F020F4883E20F481E00895843FE1F353
:1011100080E00895883EC0F3813FD1F7F5CF93FB7F
:10112000882780F90895FC01808191810E949F09A0
:101130000C947408CF93DF9300D000D00F92CDB7FA
:10114000DEB70F900F900F900F900F90DF91CF911F
:101150000895CF93DF9300D000D000D0CDB7DEB795
:1011600026960FB6F894DEBF0FBECDBFDF91CF91AC
:10117000089508950C94B9080E94BA088093BF019D
:101180000C945A0808950C94BC089091BF01892BC7
:101190000C94BC089091BF0189230C94BC089091D9
:1011A000BF0189270C94BC080C94B9080C94D4088E
:1011B0000E94D6088093BE010C945A0880E00C94DB
:1011C000D80891E001C0990F8A95EAF7892F0C940D
:1011D000D80821E030E001C0220F8A95EAF780911B
:1011E000BE01822B0C94D80821E030E001C0220F10
:1011F0008A95EAF720958091BE0182230C94D80845
:1012000021E030E001C0220F8A95EAF78091BE010B
:1012100082270C94D8089091BE01892B0C94D80891
:101220009091BE0189230C94D8089091BE01892722
:101230000C94D8080895E92FEE0FE90FEE0F8E0FEA
:10124000982F977041E001C0440F9A95EAF7869570
:101250008695869593E0899FF0011124EB54FE4F0B
:1012600030E020E070E05191DF011197CB01022EB8
:1012700002C0969587950A94E2F78170819585273B
:10128000842385278C932F5F3F4F2330310559F7F7
:101290000895E92FEE0FE90FEE0F8E0F982F97703C
:1012A00086958695869523E0829FF0011124EB5464
:1012B000FE4F50E040E080E0219130E0092E02C076
:1012C000369527950A94E2F721703327042E01C042
:1012D000220F0A94EAF7822B4F5F5F4F433051058C
:1012E00059F70895CF92DF92FF920F931F93CF93F8
:1012F000DF936C010091BE018091BF01082BC7E014
:10130000D0E010E0FC2EC8010C2E02C09595879508
:101310000A94E2F780FD0CC02197A0F7F12C8F2DE5
:10132000DF91CF911F910F91FF90DF90CF900895A3
:10133000B6018C2F0E944110019771F3F0CFCF932B
:10134000DF93EC010E947209BE01DF91CF910C94F2
:1013500041101F93CF93DF93EB019091B401992338
:1013600031F0CB01DF91CF911F910C949F0988231D
:1013700079F0CB010E947209182F682FCE010E94CC
:101380001B09BE01812FDF91CF911F910C94411059
:10139000CB010E944909182FF4CF1F93CF93DF93FD
:1013A000C091C00116E08091C1018C1304C0DF918F
:1013B000CF911F910895D0E01C9FF0011D9FF00D6B
:1013C0001124EE53FE4F40815181628173818481EB
:1013D00095810E94A9082196C770E5CF4091F2013E
:1013E0005091F3016091F4017091F5018091F60143
:1013F0009091F7010C94A908FF920F931F93CF933C
:10140000DF938091F701807FD1F48091F4018823EC
:10141000B1F08091C0011091C1016091F201709111
:10142000F301A091F501B091F601062F0723C091B9
:101430000001D091010196E0F92E181306C0DF914A
:10144000CF911F910F91FF90089590E0109711F0A8
:101450000F3F19F401968770F0CFF89E9001F99E26
:10146000300D1124F901EE53FE4F41814713F2CFA5
:1014700040814613EFCF42814111ECCF438154812B
:101480004A1B5B0B4C175D0728F78091F7018F70A3
:1014900080618093F701F901E953FE4F80818F70DD
:1014A0008061808382EF91E00E942E08DF91CF91CE
:1014B0001F910F91FF900C94CD09AF92BF92CF92E4
:1014C000DF92EF92FF920F931F93CF93DF93CDB7ED
:1014D000DEB761970FB6F894DEBF0FBECDBF8C01AB
:1014E00085E0F801DE011D9601900D928A95E1F7E5
:1014F000F801E28082EFC82E81E0D82E6091F501DC
:101500007091F6016115710509F45FC19091F201C6
:101510002091F301892F82238F3F09F456C1408126
:101520005181A380B480F090F401F501E61BF70B24
:10153000BF01E0910001F0910101FF2009F4F6C024
:101540008091F701382F307F6E177F0708F0AFC00A
:10155000311179C0FE2C251323C0941321C0E11052
:101560001FC08F7080618093F7010E94EE09C60151
:101570000E942E088091F701F80185838F2D6196D6
:101580000FB6F894DEBF0FBECDBFDF91CF911F9194
:101590000F91FF90EF90DF90CF90BF90AF900895A4
:1015A000AB2829F0842F85238F3F09F027C180E0E5
:1015B000F82FF170DF2E80FF3CC08091C001209198
:1015C000C10136E0821315C04D875E878D859E85EB
:1015D0000E949F09292F22952F702230F0F024308D
:1015E00018F59F70F1F0F8019581907FD1F4D12C1E
:1015F0001EC090E0389FF001399FF00D1124EE538A
:10160000FE4F6181651306C06081641303C062816F
:101610006E110FC001968770D5CF9F7011F088238F
:1016200031F3805E883018F3C8010E942E08FD2C2B
:10163000A5CFEE2009F4A2CF8091F70181608093BD
:10164000F701F12C9BCF251306C0941304C0F801B9
:10165000EE2009F487C0C8010E949308882319F17D
:10166000EE2009F18091F701803270F02091F201B3
:101670003091F30138872F831986BB86AA868C8721
:10168000CE0107960E942E0886E0F801A2EFB1E095
:1016900001900D928A95E1F70E94FC090E94EE09E3
:1016A000FF24F3946BCFC8010E942E08F9CF3111AB
:1016B00013C07A2DB98AA88A6E2D89890E949A084A
:1016C00082EF91E00E942E0886E0F60111928A9541
:1016D000E9F70E94EE09B5CF25130FC094130DC092
:1016E000E1100BC0F8018583C8010E942E0886E036
:1016F000F60111928A95E9F741CFC8010E9493083B
:10170000882389F2EE2079F28091F701803208F483
:10171000BBCF2091F2013091F3013A8329831B82E0
:10172000BD82AC828E83CE010196ACCF6E177F074F
:1017300008F03EC0FE2CEE2009F4B5CF25132AC0D8
:10174000941328C08091F70180FD1BC0982F907FD3
:10175000C1F0F8018583903F31F0982F907F905F22
:101760008F70892B8583C8010E942E0886E0F801BE
:10177000A2EFB1E001900D928A95E1F70E94EE0987
:10178000FDCE86E0F801A2EFB1E001900D928A95BE
:10179000E1F7F4CEC8010E949308811175CF8091C2
:1017A000F70181608093F701C8010E942E08E6CE00
:1017B0007A2DB98AA88A6E2D89890E949A0886E0B6
:1017C000F60111928A95E9F7D9CFEE2009F46BCF93
:1017D000C8010E949308F82E882309F464CF86E09C
:1017E000F801A2EFB1E001900D928A95E1F782EF46
:1017F00091E00E9467050E94FC09C0CF81E08E2520
:10180000D7CE1F93CF93DF93CDB7DEB72C970FB60C
:10181000F894DEBF0FBECDBF4F83588769877A87A4
:101820008B879C87CE0107960E945D0A882369F00A
:101830008A859B85892B39F04F815885842F852394
:101840008F3F09F071C016E05FC086E0FE01379659
:10185000DE01119601900D928A95E1F78A859B85AC
:10186000892B89F38F81988589238F3F61F320919C
:10187000C10130E0C9010196877099274091C001EC
:101880004817190671F40E9470081092C101109255
:10189000C00186E0E2EFF1E0DF011D928A95E9F7F1
:1018A000D2CF96E0929FD001939FB00D1124AE53FA
:1018B000BE4FFE01319601900D929A95E1F780930B
:1018C000C1010E94CD09BFCF819FC00111248E5359
:1018D0009E4F0E945D0A8823E9F0E091C0011E9F9F
:1018E000F0011124EE53FE4F4081518162817381DA
:1018F000848195810E94A9088091C00190E00196A1
:10190000877099278093C0018091C0019091C10197
:101910008913DACF2C960FB6F894DEBF0FBECDBF79
:10192000DF91CF911F91089569857A858B859C857C
:101930000E94A90888CF682F80910201909103012D
:101940000C94C51E682F80910201909103010C94A4
:10195000D01E80910201909103010C94DB1E8091B6
:10196000F80185958595859508958091F801877092
:1019700008959091F801977081E009F480E008954E
:1019800080911C02089590911C02892B80931C0267
:101990000895809590911C02982390931C020895BD
:1019A00010921C02089590911B02892B80931B02B8
:1019B0000895809590911B02982390931B0208959F
:1019C00010921B02089510921A0208958091F90155
:1019D000089508950C94E90C90919A0292FD08C024
:1019E0009091F901981721F08093F9010C94EA0C79
:1019F00008958091F901882329F01092F90180E07F
:101A00000C94EA0C0895E0910201F0910301809199
:101A10001C028083E0910201F0910301808190918A
:101A20001B02892B8083E0910201F09103018081E8
:101A300090911A02892B80839091F901992381F06A
:101A4000E0910201F09103018081892B80838091D4
:101A50000201909103010E94311E81110E94F90C34
:101A600080910201909103010C94DD1D08950C9466
:101A7000360D90919A0292FD10C098E0899F9001D6
:101A80001124622B6093F8010E94E9088091F8010B
:101A90008595859585950C94370D0C94E9081092E1
:101AA000F80180E00C94370D9091F801809589231E
:101AB0008093F801282F277091F4282F082E000C0E
:101AC000330B9217130659F090919A0292FD07C0BA
:101AD0008595859585950E94F4080C944F0D089581
:101AE00090919A0292FB222720F9281769F080FB37
:101AF00092F990939A028091990290919A020E9491
:101B0000BB0D82E00C94540D089580919A0282FBE3
:101B1000882780F991E089270C94700D81E00C945E
:101B2000700D80E00C94700D6FEF7FEF90E080E01F
:101B30000C94E22790E080E00E94BE27893E9E4FF1
:101B400011F40C94301580E0089582E090E00C943C
:101B5000B62783E090E00C94B627CF9384E090E022
:101B60000E94B627C82F82E290E00E94B627982FE5
:101B70008C2FCF910895CF93C92F682F84E090E0E8
:101B80000E94C4276C2F82E290E0CF910C94C4276E
:101B9000AB01BC018FE090E00C94D627AB01BC01F7
:101BA00083E190E00C94D62760E070E0CB010C94C8
:101BB000CE0D60E070E0CB010E94C80D0C94D40DF6
:101BC00069EE7EEF90E080E00E94E22760E082E034
:101BD00090E00E94C42760E083E090E00E94C42768
:101BE0001092BF0160E084E090E00E94C42760E0B2
:101BF00082E290E00E94C42760E085E090E00E94CD
:101C0000C42760E086E090E00E94C4276FEF87E081
:101C100090E00E94C42740E050E0BA0188E090E0E4
:101C20000E94D62760E08DE090E00E94C42740E04B
:101C300050E0BA0188E190E00E94D62760E087E199
:101C400090E00E94C42740E050E0BA018CE190E0AF
:101C50000E94D62770E060E080E290E00E94E227D8
:101C600040E050E0BA0188E190E00E94D62780E091
:101C70000E9449150E946F150C94D90D0C94E00D2B
:101C8000682F8EE090E00C94C4270E94891F609317
:101C9000290270932A0280932B0290932C02609366
:101CA00025027093260280932702909328020895BC
:101CB0000E94891F6093290270932A0280932B024D
:101CC00090932C026093210270932202809323024E
:101CD00090932402089585B7806885BF85B7806892
:101CE00085BF0895089508950C94720E08950C947C
:101CF000760E0E946B0E8FE191E10E94C71D0E943B
:101D0000730E0C94740E81E008950C94830E089564
:101D100008950E94870E0C94880E0E94741F0E94E2
:101D20007E150E94FD1180E00E94B5160E947D1B69
:101D30000C94770E9F92AF92BF92CF92DF92EF9268
:101D4000FF920F931F93CF93DF93CDB7DEB72A9700
:101D50000FB6F894DEBF0FBECDBF0E941212C82E80
:101D600081110E94450E8EE1A82E82E0B82E10E06F
:101D700000E0902E802F0E945911E82EF501F1907D
:101D80005F01F81609F45CC080912D0281FD0E946C
:101D90005F118F2D8E25D12CFF24F394982F9F2136
:101DA00009F449C00E94850E882399F0DE829F8243
:101DB000EF2081E009F480E088870E947D1F816028
:101DC000782F9A8789874E815F8168858A850E94EE
:101DD0002905F801E25EFD4F8081F826F0820E941D
:101DE000901B182F81110E94580E0E948D18C1104F
:101DF00001C011110E9454170E9416140E94D11D97
:101E000090911D02891799F10E94D11D80931D02A6
:101E10002A960FB6F894DEBF0FBECDBFDF91CF91EB
:101E20001F910F91FF90EF90DF90CF90BF90AF90F8
:101E30009F900C942105D394FF0CF6E0DF12AECFF7
:101E40000F5F1F4F0330110509F093CF8FEF898388
:101E50008A831B820E947D1F8160782F9D838C83E3
:101E600049815A816B818D810E942905B8CF2A96BC
:101E70000FB6F894DEBF0FBECDBFDF91CF911F919B
:101E80000F91FF90EF90DF90CF90BF90AF909F9019
:101E90000895CF93DF930E944510EC01811521E551
:101EA000920708F042C0811530E5930708F09DC005
:101EB000883E910530F5803E910508F092C0883A41
:101EC000910588F4853A910508F084C08130910528
:101ED00009F487C0009709F484C0049708F081C012
:101EE000D0E0C0E07EC08F3B9105D0F7C85AD0E06B
:101EF000CC0FDD1FCF5ADE4F0990D881C02DD4649E
:101F000070C08115904250F4C11581E0D80708F0E7
:101F100068C0C03FD10520F3D06563C0C11590E40F
:101F2000D907F0F2DF70D06A5CC0811525E5920711
:101F300000F5811534E5930708F08BC0811543E562
:101F4000940708F073C0C11582E5D80708F469C08A
:101F5000CE018370992721E030E002C0220F331FA9
:101F60008A95E2F7C695C69580E2C89FE0011124E4
:101F700054C0C11599E5D907A8F4C11528E5D207C1
:101F800008F06CC0C11536E5D30708F0A9CF8C2F37
:101F90000E94DC10C82FD0E0DC2FCC27CC27DF71CB
:101FA000D0621FC0C1154AE5D40708F45CC0CE0159
:101FB00090568115904208F093CF8D2F8F710E941B
:101FC000DC1090E0982F882788279F719C012C2B8C
:101FD000E901E6CFC55AD0E0C158DE4FC881D0E054
:101FE000D064CE01DF91CF910895E4E09695879576
:101FF000EA95E1F783702C2F26952695237040E211
:10200000249F90011124382B8C2F8370C1E0D0E0E5
:1020100002C0CC0FDD1F8A95E2F7C22BD32BDC6800
:10202000E0CFDC2FCC27C16FD06ADBCF837099273C
:1020300021E030E002C0220F331F8A95E2F7C695F7
:10204000C69590E2C99FE0011124C22BD32BDA6818
:10205000C8CFD82FCC27C46FD06AC3CFDC2FCC27F2
:10206000C06FD06ABECF8C2F8F700E94DC1034E01E
:10207000D695C7953A95E1F7CF709C2FEC01D069C2
:10208000B0CF0E94A91A0C94490F82389105B1F182
:10209000B0F48133910509F475C048F48932910593
:1020A00009F469C08A32910509F473C00895853333
:1020B000910509F459C08933910501F10895833ED2
:1020C0009105A9F138F4803E9105F9F0823E910521
:1020D00049F10895863E9105A9F1873E9105C9F120
:1020E000843E910519F520919A0221FF1FC080912D
:1020F000990284FD14C087EE90E008952091990222
:102100002370A1F080EE90E008952091990220FDC7
:1021100047C030919A0230FF09C024FF44C090E0CC
:1021200080E004C02091990222FDF7CF089520910C
:10213000990222FD3BC030919A0230FDE3CF24FF8B
:10214000F5CFEDCF2091990223FFF0CF24FDE7CF0B
:10215000D2CF2091990223FD2CC030919A0231FFF9
:10216000EECF84EE90E008952091990225FFDECF16
:1021700089E290E008952091990225FFD7CF85E369
:1021800090E008952091990226FFD0CF8AE290E056
:1021900008952091990226FFC9CF81E390E0089528
:1021A00089E390E0089583EE90E0089582EE90E058
:1021B000089586EE90E008959091990292FF06C0EE
:1021C000282F28712830F9F4877F846093FF06C098
:1021D000282F28712831F1F4877E846120919A029A
:1021E00020FF06C0382F38713830D9F4877F8160DE
:1021F00021FF06C0282F28712831D1F4877E816104
:1022000094FD877E0895282F24712430F9F68B7F62
:102210008860DCCF282F2471243101F78B7E886100
:10222000DDCF382F3171313019F78E7F8860E0CFE4
:10223000282F2171213121F78E7E8861E1CF80E046
:1022400008950C94940D0E9412128FE39CE901975B
:10225000F1F700C000000E94121280E00E945911A4
:1022600080FF04C00E9421110C94C81F08950C9493
:1022700023110E949A0D811102C00E943E0E0E94FD
:10228000A50D80932D020E94AD0D90939A0280932C
:1022900099020E9437110E94A90D0E94C3088091E3
:1022A000BE010C94D60808950C94531108950C9413
:1022B0005611E82FF0E0E256FD4F80810895089511
:1022C00080EA8A95F1F7089500C008950C94601192
:1022D000F894E82FE295EF70F0E031A1282F2F70ED
:1022E00081E090E001C0880F2A95EAF7982F909539
:1022F000932391A392A1892B82A378940895CF93DD
:10230000DF9386EC0E94681187EF0E94681187E6D0
:102310000E946811C2E8D1E089918F3F11F00E94BC
:10232000681181E0C838D807B9F7DF91CF910895D7
:10233000CF92DF92EF92FF920F931F93CF93DF9391
:10234000EC01D62E062F10E0C80188579E4F7C0165
:10235000FC0180818F3F09F445C0F894E82FE29595
:10236000EF70F0E091A18F7021E030E001C0220F0A
:102370008A95EAF7892F822B81A382A120952823B1
:1023800022A378940E946411E2E8F1E048E851E069
:1023900031E0C12C21912F3F71F1A22FA295AF7096
:1023A000B0E090968C9190E02F7002C09595879543
:1023B0002A95E2F780FD1FC0832FC82A330F4E17DE
:1023C0005F0741F7F70180818F3F11F00E9468118C
:1023D00061E0C11001C060E08D2D0E946611C00F48
:1023E000D11FC882DF91CF911F910F91FF90EF9085
:1023F000DF90CF90089580E0E0CF0E947F1183E0CE
:10240000EEE9F2E0DF01982F1D929A95E9F7EBE9EA
:10241000F2E0DF011D928A95E9F783E00E945512F0
:102420000C94C5031F93CF93DF9300D00F92CDB7C9
:10243000DEB719821A821B8260E0CE0101960E94EB
:10244000981161E0CE0101960E94981162E0CE01E0
:1024500001960E94981143E050E0BE016F5F7F4FEC
:102460008BE992E00E94A92711E0009709F410E09F
:10247000892B49F089819A81AB8180939B0290934B
:102480009C02A0939D02212F43E06EE972E08BE94C
:1024900092E00E9456120E94CB03812F0F900F9062
:1024A0000F90DF91CF911F9108950895FF920F93A0
:1024B0001F93CF93DF93F82E092F162FD72FC42FFA
:1024C000222349F081E0809330020E947D1F909387
:1024D0002F0280932E02809130028823A1F08091F8
:1024E0002E0290912F020E94951F059760F0EF2D0C
:1024F000F02FA12FBD2FCE0FDF2FD11DEC17FD0721
:1025000041F410923002DF91CF911F910F91FF9013
:10251000089581918D93F2CF0E94C3210E948D0E68
:102520000C94CF210E94D3210E949A0E0C94ED218D
:102530000E94071F0E94AA210E94790E0E948C12FD
:102540000E9492120E94890EFBCF8091370280FF79
:1025500012C06091090185E0689FB0011124759552
:1025600067957595679560387105A8F561157105D2
:10257000A1F1862F089581FF09C06091090185E0CE
:10258000689FB001112475956795EDCF60910901A1
:1025900082FD0AC0809136028823D1F09091080113
:1025A00060910901891728F085E0689FB001112426
:1025B000DACF869FB001112485E0869F9001879F26
:1025C000300D1124692F70E0C9010E948827CBCFFC
:1025D00065E070E0CECF8FE7089581E008958091A7
:1025E000370280FF0CC06091050170E0759567951A
:1025F000759567956115710549F1862F089581FFDD
:1026000006C06091050170E075956795F3CF609104
:10261000050182FD0BC0909135029923A1F06091D4
:10262000040180910501961738F0682F70E060383A
:10263000710500F38FE70895899FC001112470E0B0
:102640000E948827F4CF61E070E0D7CF81E0089541
:10265000803F31F40E94A512819580933B0208953A
:10266000813F19F40E94A512F8CF823F31F40E94F5
:10267000A512819580933A020895833F19F40E9430
:10268000A512F8CF893F29F40E94EF1280933C02F3
:1026900008958A3F21F40E94EF128195F7CF8B3F76
:1026A00031F40E94EF12819580933D0208958C3F92
:1026B00019F40E94EF12F8CF9CE0980F953070F457
:1026C000845F990B21E030E001C0220F8A95EAF780
:1026D00080913902822B8093390208958D3F31F425
:1026E0008091370281608093370208958E3F21F4F4
:1026F000809137028260F7CF8F3FB9F78091370220
:102700008460F1CF40913A02803F59F480913B02BE
:1027100087FF0DC010923B0241110BC01092360290
:1027200008C0813F81F480913B0218169CF344233A
:1027300081F080913C0290913D02892B09F05AC0B2
:10274000109235020895823F49F447FFF0CF10926E
:102750003A0280913B028111ECCFE0CF833F19F424
:102760001416ACF3E4CF90913C02893F29F419167A
:10277000F4F610923C02DBCF8A3F19F497FFD7CFD3
:10278000F8CF90913D028B3F29F497FFD0CF109264
:102790003D02CDCF8C3F19F41916CCF3C8CF9CE085
:1027A000980F953090F4845F990B21E030E0B901E7
:1027B00002C0660F771F8A95E2F7CB018095909152
:1027C0003902892380933902B2CF8D3F31F4809151
:1027D00037028E7F80933702AACF8E3F21F48091FB
:1027E00037028D7FF7CF8F3F09F0A1CF809137025D
:1027F0008B7FF0CF08950E947D1F9C0190913A023B
:1028000080913B02982B21F03093340220933302C5
:1028100090913C0280913D02982B21F0309332023E
:102820002093310288E392E00C94F71DEF92FF921F
:102830000F931F93CF93DF9300D000D000D0CDB77C
:10284000DEB786E0E8E3F2E0DE01119601900D923A
:102850008A95E1F7E0903A02F0903B0200913C0249
:1028600010913D0210923A0210923B0210923C02EB
:1028700010923D028E2D8F2991F08091330290911C
:1028800034020E94951FAC0190913602992309F4FD
:102890003FC080910A018417150608F447C0802FB5
:1028A000812B91F080913102909132020E94951F0C
:1028B000AC0190913502992309F477C0809106010B
:1028C0008417150608F47FC080913A0290913B026C
:1028D000892B90913C02892B90913D02892B11F01C
:1028E0000E94FB1386E0FE013196A8E3B2E001905E
:1028F0000D928A95E1F726960FB6F894DEBF0FBECB
:10290000CDBFDF91CF911F910F91FF90EF90089570
:1029100020910B018AE0289F90011124241735078C
:1029200008F0BDCF9F5F9093360202C09F3FD1F762
:10293000EE2059F00E94A5129FEF1E140CF491E0B6
:10294000899F802D112480933A02FF2059F00E9424
:10295000A5129FEF1F140CF491E0899F802D112484
:1029600080933B0230913A02332309F498CF2091AF
:102970003B02222309F493CF45EB3403C001112419
:10298000992359F090933A0245EB240390011124C6
:10299000332339F030933B0282CF81E080933A02B7
:1029A000F3CF81E080933B027ACF209107018AE048
:1029B000289F900111242417350708F085CF9F5FC9
:1029C0009093350202C09F3FD1F7002359F00E9437
:1029D000EF129FEF10160CF491E0899F802D1124C7
:1029E00080933C02112359F00E94EF129FEF1116C1
:1029F0000CF491E0899F802D112480933D02309149
:102A00003C02332309F460CF20913D02222309F4D4
:102A10005BCF45EB3403C0011124992359F0909307
:102A20003C0245EB240390011124332339F0309309
:102A30003D024ACF81E080933C02F3CF81E0809356
:102A40003D0242CF86E0E8E3F2E0DF011D928A9585
:102A5000E9F710923602109235021092370208956B
:102A600083E290E00E94B627823289F484E290E00B
:102A70000E94B627823059F485E290E00E94B62782
:102A800091E0833209F090E0892F8170089580E011
:102A9000FCCFCF93C82F6FEF811162E283E290E009
:102AA0000E94C4276FEFC11162E084E290E00E94AF
:102AB000C4276FEFC11163E285E290E0CF910C94DF
:102AC000C427089586E290E00E94B627682F70E040
:102AD00090E080E0089586E290E00C94C42780E0C6
:102AE0000E94491560E070E0CB010E946B150E94C6
:102AF000231A0E940D1B81E00C9449150E94611558
:102B00000E943015811102C00C946F150895CF9367
:102B1000FB01C281CC2309F19C0122513F452031A8
:102B2000310520F582510E941D1BC0E08C2FCF91F2
:102B3000089581E00E94E90843E062E081E00E949C
:102B4000BC03F3CF81E00E94F40843E062E081E03F
:102B50000E94BC03EBCF82E0F6CF8031FFE59F07F8
:102B600089F381319F45B9F3C1E0E0CF8031EFE5D2
:102B70009E07F9F281319F45C9F682E0DBCF2FEF46
:102B8000FC01208308951F93CF93DF93EC01162F50
:102B9000E881E150E33108F059C0F0E0EC5EF74D18
:102BA0000C949C27198289E08A83612FCE01DF91E2
:102BB000CF911F910C94832089818230D1F0833092
:102BC00059F08130C9F40E94891F0E94A2276A83AC
:102BD0007B838C839D83E9CF80E00E9459118A8397
:102BE00081E00E9459118B8382E00E9459118C83ED
:102BF000DCCF0E946215E9CF612FCE010E94BF1584
:102C0000D4CF89818230C1F76A817B818C819D819B
:102C10000E94A2270E946B15C8CF4B816A818981CF
:102C20000E94F5199827892798279D838C83BDCF0B
:102C30002C813D813227232732274B816A8189816C
:102C40000E940E1AB2CF0E94231AAFCF8FEF888353
:102C5000ACCF0E94B61A8983A8CF0E94B81A9827D1
:102C6000892798279A838983A0CF6B8170E0898117
:102C70009A81AE014C5F5F4F9827892798270E9461
:102C8000BB1A93CF6B8170E089819A81AE014C5F52
:102C90005F4F9827892798270E94E21A86CF0E94C3
:102CA0000D1B83CF0E94E319D6CF6B8170E0898121
:102CB0009A81AE014C5F5F4F9827892798270E9421
:102CC0005B1A73CF6B8170E089819A81AE014C5F92
:102CD0005F4F9827892798270E94801A66CFCF9246
:102CE000DF92EF92FF920F931F93CF93DF936C01CC
:102CF0007B0164E670E088E70E94C61CEC0197FD4A
:102D000012C010E000E0F601E00FF11F849164E6CC
:102D100070E00E94401DEC01892B29F40F5F1F4FCA
:102D20000E151F0581F70E94C31DCE01DF91CF91C3
:102D30001F910F91FF90EF90DF90CF90089508952D
:102D4000E1EAF2E080E092E0DF019C011D92215077
:102D50003040E1F7F093A604E093A5048FEF9FEFD6
:102D6000909364028093630208950E949F160E94CC
:102D70003E0380935F0280FD0FC080E880935E0277
:102D80000E94C01C6DE070E083E094E00E946F162A
:102D9000892B21F080E0089580E2F0CF80915F02DE
:102DA00063E070E081FD26C080E094E00E946F1631
:102DB000892B81F76DE070E080EF93E00E946F1641
:102DC000892B41F70E94891F605A75418F4F9F4F91
:102DD0006093A1047093A2048093A3049093A4042D
:102DE0000E94A01681E0809362028093610210929B
:102DF000600208958DEF93E0D9CF20915E0236E016
:102E0000839FC0011124629F800D911D11248115A3
:102E100022E0920714F090E080E08F559D4F909350
:102E2000A6048093A5040895CF93DF932091A50471
:102E30003091A604215A3240A901460F571F413054
:102E4000524020F060E072E0621B730B409163021D
:102E500050916402FC01C901620F731FC1E0D0E010
:102E60008617970738F05093640240936302DF910E
:102E7000CF9108952491DC01AF55BD4F3C9132179D
:102E800081F02C939C01A5E036952795AA95E1F752
:102E9000DE0102C0AA0FBB1F2A95E2F79D014A2B53
:102EA000532B01963196DCCF80916202811103C0D1
:102EB0008091610208950E94891F605A75418F4F69
:102EC0009F4F6093A1047093A2048093A3049093F6
:102ED000A404809161028111EBCF62E070E08EEE7C
:102EE00093E00E946F16892B19F781E080936102AD
:102EF000DFCF2F923F925F926F927F928F929F923D
:102F0000AF92BF92CF92DF92EF92FF920F931F93F7
:102F1000CF93DF9380916202882369F0209163024E
:102F2000309164022115310531F08091600261E039
:102F300070E0882399F0DF91CF911F910F91FF905E
:102F4000EF90DF90CF90BF90AF909F908F907F9049
:102F50006F905F903F902F9008958F5F082F10E043
:102F60001B01082E02C0220C331C0A94E2F7A901AF
:102F700042215321452B89F390915F0290FD44C07B
:102F80008295880F807680930E019801369527955B
:102F90003695279520931101815E80930F01109241
:102FA000120124E630E047E050E06CE071E088E791
:102FB0000E946F1D892B09F0BECFA80125E0440FA8
:102FC000551F2A95E1F780915F0280FD2BC04F5578
:102FD0005D4F04E610E020E230E060E488E70E9404
:102FE000961D892B09F0A7CF0E945417E101C095C7
:102FF000D0958091630290916402C823D923D09325
:103000006402C093630297CF880F880F880F809364
:103010000E0110921101895F80930F0183E080936C
:103020001201BFCFEEE3F2E080E2DF011D928A954C
:10303000E9F7AFE8B1E00BE811E083E9C82E81E0E1
:10304000D82E97E0592E772473948D91E801299119
:103050008E01240F352F311D2F553D4FE82FF0E005
:10306000E25CFD4F90E080E0652C681A872C082E0A
:1030700001C0880C0A94EAF77901A12CE701B99004
:103080007E01B820662D6A196770962E062E000CF8
:10309000770BDB2D01C0DD0F9A94EAF771956195EE
:1030A00071096770772701C0B6946A95EAF7BD2A5F
:1030B0006081962E9B289082A39468E0A612DECFB2
:1030C000019631968830910579F6CA16DB0609F02B
:1030D000BCCF04E610E020E230E04EE352E07DCFCA
:1030E0008091610290916202911103C091E0892761
:1030F0000895882369F062E070E08CEE93E00E940E
:103100006F16892B19F08091610208951092610267
:1031100080916102EBCF0C9436030F931F93809143
:103120006202882319F160E080E00E94FD160E948F
:103130008B180E947917809161028823B9F00E9450
:10314000891F0091A1041091A2042091A304309141
:10315000A404601B710B820B930B6F3F7F4F8F4F4B
:103160009F4720F41F910F910C9470181F910F919D
:103170000895CF93DF93EC01FB018281882309F44A
:1031800020C1C330FDE5DF07C8F5CA3F9CE5D9077C
:1031900030F49E0122503C452431310598F50E94BF
:1031A000AD0D90939A0280939902C031FCE5DF0740
:1031B00009F4E0C008F061C0C8309CE5D90709F403
:1031C000CBC088F5C430FCE5DF0709F4B3C0E8F4F0
:1031D000C2309CE5D90709F4A7C0809199028260AA
:1031E000C330DC4509F4A3C08091990290919A0202
:1031F0000E94BB0D0E94700880E004C0C136EDE55E
:10320000DE0769F2DF91CF91089580919902806184
:10321000C630FCE5DF0709F48AC008F48FC080914E
:103220009902806284C0809199028D7FCC309CE5A8
:10323000D90709F47CC070F4809199028C60CA307F
:10324000FCE5DF0709F473C008F48AC08091990295
:103250008E7F6DC080919902877FCE309CE5D90723
:1032600009F465C0809199028B7FCF30DC4508F46A
:103270005EC0809199028F7E5AC0CC3FFCE5DF078B
:1032800009F474C040F5C4319CE5D90709F48AC03B
:1032900058F4C231FCE5DF0709F474C008F46EC0CD
:1032A00080919902837F43C0CA3F9CE5D90709F406
:1032B00049C008F04DC0C531DC4509F095CF80917B
:1032C000990282FB992790F921E0922790FB82F9DD
:1032D00090FB83F92CC0C1158DE5D80709F458C0BF
:1032E00088F480919A028360CE3FECE5DE0769F1B5
:1032F00080919A028D7FCF3FDC4538F180919A0210
:103300008C7F23C0C2308DE5D80709F458C008F47B
:1033100052C0C136DD4509F067CF90919902892FDF
:103320008F7E94FF806103C08091990281608093B9
:1033300099025ACF809199028460F9CF80919902C5
:103340008860F5CF80919A02816080939A024CCF79
:1033500080919A028260F9CF809199028064E7CFD0
:103360000E947008809199028068E1CF80919A0252
:103370008E7FEBCF809199028F7DD9CF809199027A
:103380008F7BD5CF0E947008809199028F77CFCF25
:1033900080919A02982F909591708E7F892B90FB47
:1033A00081F9D3CF0E94700890919902892F97FBE1
:1033B00087F98058BCCF81E00E94400E15CF80E095
:1033C000FBCF81E01FCF84E0089550E0440F551FEC
:1033D0009CE0699F400D511D112494E2899F400D8E
:1033E000511D1124CA01879608950F931F93CF93FF
:1033F000DF930E94E5198C010E94B627C82FD0E008
:10340000DC2FCC27C80101960E94B6279E01282BED
:10341000C901DF91CF911F910F9108950F931F93D1
:10342000CF93DF93122F032F0E94E519EC01602F39
:103430000E94C427612FCE010196DF91CF911F9189
:103440000F910C94C427AF92BF92CF92DF92EF926C
:10345000FF921F93CF93DF938CEAC82E82E0D82E81
:10346000D0E07601C0E014C0F50125913491412FE0
:103470006C2F8D2F0E940E1A82E0A80EB11C1F5FC8
:10348000163091F78CE0E80EF11CCF5FC33019F0D5
:10349000570110E0E9CFDF5F84E2C80ED11CD430C1
:1034A00001F7DF91CF911F91FF90EF90DF90CF90C8
:1034B000BF90AF900895EF92FF920F931F93CF9319
:1034C000DF93EC018A017C01E60EF71ECE018796A0
:1034D000CE15DF0539F4DF91CF911F910F91FF9049
:1034E000EF900895C039D10540F40E94B627F80145
:1034F00080830F5F1F4F2196E9CFF8011082F9CF2B
:10350000CF92DF92EF92FF920F931F93CF93DF93AF
:103510007C016A018C01060F171FEC01CE01879612
:10352000C017D10749F4DF91CF911F910F91FF9000
:10353000EF90DF90CF900895C039D10540F4FE019F
:10354000EE19FF09EC0DFD1D60810E94C427219634
:10355000E5CF462F843038F4733028F4663018F401
:10356000672F0C94F51990E080E0089580E10895AC
:1035700089E493E00895EF92FF920F931F93CF9306
:10358000DF93EC018A017C01E60EF71ECE0189541F
:103590009F4FCE15DF0539F4DF91CF911F910F9129
:1035A000FF90EF900895C93423E0D20740F40E94C1
:1035B000B627F80180830F5F1F4F2196E7CFF801F0
:1035C0001082F9CFCF92DF92EF92FF920F931F9369
:1035D000CF93DF937C016A018C01060F171FEC016A
:1035E000CE0189549F4FC017D10749F4DF91CF9185
:1035F0001F910F91FF90EF90DF90CF900895C93405
:1036000023E0D20740F4FE01EE19FF09EC0DFD1D89
:1036100060810E94C4272196E3CFCF93DF93C7EB4D
:10362000D0E060E0CE010E94C4272196C11584E05D
:10363000D807B9F7DF91CF910895DF92EF92FF920B
:103640000F931F93CF93DF9300D000D0CDB7DEB799
:10365000F82E8FE08F1540F08FEF93E00E94B62791
:1036600007EB10E08823C1F00F900F900F900F90A0
:10367000DF91CF911F910F91FF90EF90DF90089510
:10368000011584E0180781F3C8010E94B627811153
:1036900001C0FA940F5F1F4FF110F2CF19821A8206
:1036A0001B821C82DD24D39478018FEFE81AF80A7C
:1036B000C8010E94B62789831A828823A9F29FEF46
:1036C000980F933078F48A83D9820E5F1F4FC70119
:1036D0000E94B6278B83882339F2CE0101960E947F
:1036E0001605E2CF8701F9CF8FE891E00197F1F756
:1036F00000C0000008950C94400322982A9A239851
:103700002B9A0E94741B83B182FB882780F91B9936
:1037100005C090E0892B80936702089592E0FACF6C
:10372000E0916702EE0FEE0FE093670243B142FBB8
:10373000882780F943B143FB222720F943FF02C0C9
:1037400022E030E0822BE82BE0936702EF70F0E09C
:10375000ED56FE4F808190916602890F809366023C
:1037600020E0823054F0809165028F5F8093650283
:1037700060E080E00E947B1B21E0809166028F3F29
:1037800054F48091650281508093650261E080E08D
:103790000E947B1B21E080916602082E000C990B91
:1037A00062E070E00E94882780936602822F08956D
:1037B000CF93DF93EB0186319C4511F50E94C00C3D
:1037C0009A81992399F08A7A91E009F490E0909394
:1037D0006802811109C089E20E949B0C0E94030DBE
:1037E00080E0DF91CF91089585E3F6CF8091680264
:1037F000811104C089E20E94A20CF0CF85E3FBCFC7
:1038000081E0EFCF0F931F93CF93DF93C42FD22F7D
:10381000FC0182818823C9F040936B020E947D1FC6
:1038200090936A028093690280E28C0F883008F0DE
:1038300050C0C77081E001C0880FCA95EAF7DF91D8
:10384000CF911F910F910C94080610916B021413E5
:1038500035C08091690290916A020E94951F883C50
:10386000910560F5C0E2CD0F1D17B9F080E2810F20
:10387000883040F4177081E001C0880F1A95EAF78C
:103880000E940F06C83048F481E09D2F977001C058
:10389000880F9A95EAF70E940806802F0E9400067A
:1038A000C830B8F4D77081E001C0880FDA95EAF724
:1038B000DF91CF911F910F910C940F0680E28C0F36
:1038C000883038F4C77081E001C0880FCA95EAF7E4
:1038D000EFCFDF91CF911F910F9108950F939C012E
:1038E000CB01233F4CE5340759F1A8F4283DFCE512
:1038F0003F0701F1293D4CE53407D1F1273D3C4517
:1039000091F406E221EE41EE67ED7CE50E94021C97
:1039100080E00F910895253FFCE53F07E9F0B0F006
:10392000263F3C45F9F0FC018281882339F1109251
:103930006B02EFCF07E225EE45EE68ED7CE5E6CFC2
:1039400006E221EE40EE63EF7CE5E0CF07E225EEF4
:1039500044EE64EF7CE5DACF06E221EE42EE65EF5D
:103960007CE5D4CF07E225EE46EE66EF7CE5CECFD0
:1039700008E221E045EE69ED7CE5C8CF81E0C9CFE2
:103980001092B9008CE08093B80008959F92AF9296
:10399000BF92CF92DF92EF92FF920F931F93CF933C
:1039A000DF93B82EEB010E947D1F6C01EE24E3949F
:1039B000F12CC431D10560F025E0E22EF12CCF3F8F
:1039C000DC0731F0CE0164E170E00E9474277B01D6
:1039D00084EAA82E94E8992E1092BC00A092BC0014
:1039E0000E947D1F8C018091BC0087FF0DC08091DB
:1039F000B900887F883039F18091B900887F8031A3
:103A000011F10FEF1FEF09C00E947D1F801B910B6A
:103A10008E159F0540F30EEF1FEFCF3FDC07E1F25D
:103A2000C6010E94951F8C179D07B0F2C801DF9157
:103A3000CF911F910F91FF90EF90DF90CF90BF90AB
:103A4000AF909F900895B092BB009092BC000E94EE
:103A50007D1F8C018091BC0087FF0AC08091B90056
:103A6000887F883111F0803461F610E000E0DECF0D
:103A70000E947D1F801B910B8E159F0558F3CBCFA5
:103A80000F931F93CF93DF93EB018093BB0084E8E8
:103A90008093BC000E947D1F8C018091BC0087FF39
:103AA00011C02091B900287F81E090E0283211F404
:103AB00090E080E0919581959109DF91CF911F91E0
:103AC0000F910895CF3FDC0741F30E947D1F801BBB
:103AD000910B8C179D0708F38EEF9FEFEECFCF92DF
:103AE000DF92EF92FF920F931F93CF93DF936B01BF
:103AF0008A017901B9010E94C61CE6010C0D1D1D49
:103B0000C017D10761F424E92093BC00DF91CF9165
:103B10001F910F91FF90EF90DF90CF90089597FD48
:103B2000F2CFB70189910E94401DEACFCF92DF9278
:103B3000EF92FF920F931F93CF93DF93C62F6A01EB
:103B40007901B8010E94C61C97FD0CC0B8018C2FEA
:103B50000E94401DE601EC0CFD1CCE15DF0511F0A6
:103B600097FF0CC024E92093BC00DF91CF911F91F7
:103B70000F91FF90EF90DF90CF900895B801899159
:103B80000E94401DEACF84E98093BC000895909381
:103B9000B3018093B20108959093710280937002F3
:103BA0000895E0917002F0917102309721F0019038
:103BB000F081E02D099480E00895E0917002F09189
:103BC0007102309799F020911F01222359F0209122
:103BD000990227FF07C0DC012C9111962C931197B5
:103BE00026E02C930280F381E02D09940895E09162
:103BF0007002F0917102309739F022E0DC012C93D1
:103C00000480F581E02D0994089520916E02309191
:103C10006F022817390771F090936F0280936E023C
:103C2000E0917002F0917102309721F00680F781E7
:103C3000E02D0994089520916C0230916D022817AF
:103C4000390771F090936D0280936C02E0917002DD
:103C5000F0917102309721F00084F185E02D0994F4
:103C60000895FC01329680911F01882321F08091F4
:103C700099029EE187FF96E080E0915008F4089554
:103C800021912223D1F38F5FF8CF662301F1209198
:103C90001F012223F1F02091990227FF1AC0462F1D
:103CA0004695469546954E3190F4677021E030E098
:103CB00002C0220F331F6A95E2F7840F911DFC01A9
:103CC000828190E02823392381E0232B69F480E06E
:103CD0000895FC01329608962191261721F0E817E5
:103CE000F907D1F7F4CF81E008959C01FC013296E9
:103CF0009FEF80E04191461751F09F3F19F4411129
:103D000001C0982F8F5F8630A9F79F3F09F408956F
:103D1000290F311D97FD3A95F90162830895FC0141
:103D2000329608962191261303C0DF0111971C9249
:103D3000E817F907B9F70895E62FE695E695E695B1
:103D4000EE3168F4E80FF92FF11D677021E030E0E3
:103D500001C0220F6A95EAF78281822B828308953F
:103D6000E62FE695E695E695EE3170F4E80FF92F2B
:103D7000F11D677021E030E001C0220F6A95EAF77B
:103D80002095828128232283089520911F012223D8
:103D900029F02091990227FD0C949C1E0C94751E0D
:103DA00020911F01222329F02091990227FD0C94D4
:103DB000B01E0C948F1EFC01329680911F01882347
:103DC00051F08091990287FF06C08EE1DF011D92BC
:103DD0008A95E9F7089586E0F9CF08950C94ED1ED1
:103DE000811105C081E0809372020C94EE1E82E086
:103DF000FACF83E0809372020C94EE1E0C94F01EB6
:103E000081E0809372020C94EE1E0C94001F0895C2
:103E10008091AF04843031F10E94D103109273027B
:103E200088E190E020E40FB6F894A89580936000B4
:103E30000FBE2093600083B7817F846083BF83B708
:103E4000816083BF7894889583B78E7F83BF0FB6D8
:103E5000F894A8958091600088618093600010922A
:103E600060000FBE089508950895CF930E94331FF8
:103E70000E9412120E94341FC0E08C2F0E94591120
:103E8000811105C0CF5FC330C1F7CF91089581E0A4
:103E9000FCCF0E9470080C9442041F921FB61F9220
:103EA00011248F939F93AF93BF93809173028111DD
:103EB00013C08091A7049091A804A091A904B09187
:103EC000AA044196A11DB11D8093A7049093A80454
:103ED000A093A904B093AA04BF91AF919F918F9131
:103EE0001F901FBE1F90189582E084BD93E095BD82
:103EF0009AEF97BD80936E0008952FB7F894809144
:103F0000A7049091A804A091A904B091AA042FBF7E
:103F100008952FB7F8946091A7047091A804809138
:103F2000A9049091AA042FBF08959C014FB7F8945B
:103F30008091A7049091A804A091A904B091AA042B
:103F40004FBF821B930B089578941F921FB61F9248
:103F500011248F939F93AF93BF938091A704909167
:103F6000A804A091A904B091AA040196A11DB11DB5
:103F70008093A7049093A804A093A904B093AA04E3
:103F8000BF91AF919F918F911F901FBE1F90189569
:103F900081E08093E00080E28093D8001092C90015
:103FA0008FE19EE40197F1F700C0000087E090EBFD
:103FB000DC018093B8049093B904A093BA04B09341
:103FC000BB0488E19CE00FB6F894A895809360004C
:103FD0000FBE90936000FFCF8091970208950895DF
:103FE0009C0184E08093E9009FEF8091E80091506C
:103FF00085FD06C085ED8A95F1F700009111F5CF9A
:104000008091E80085FF0CC050E040E066E070E081
:10401000C9010E9494228091E8008E778093E80085
:104020000895CF93DF93EC0180911F018823B1F1B4
:104030008091990287FF32C060E284E08093E900BA
:104040008FEF9091E800815095FD06C095ED9A950F
:10405000F1F700008111F5CF8091E80085FF1BC0CA
:1040600080911F0170E050E040E0811104C050E0F9
:1040700040E068E070E0CE010E9494228091E80068
:104080008E778093E80080E2FE01A7E7B2E001901E
:104090000D928A95E1F7DF91CF91089568E081E074
:1040A000CDCF8093740270937602609375028091F5
:1040B000AF048430F9F48093E9008FEF9091E80029
:1040C000815095FD06C095ED9A95F1F7000081119C
:1040D000F5CF8091E80085FF0DC050E040E063E03F
:1040E00070E084E792E00E9494228091E8008E774D
:1040F0008093E8000895BC0184E00C945120BC0139
:1041000083E00C945120CF93FC01603221F5809123
:10411000AF04843001F5C091E900CF702091EC002C
:10412000922F917020FD90E8C92B82E08093E900E6
:104130008091E80080FF0CC050E040E060E270E059
:10414000CF010E9494228091E8008E778093E8004E
:10415000CF70C093E900CF9108958091AE04811192
:1041600009C00E9473240E94D0248091E2008460E0
:104170008093E20008951092AE0408950C94001FFD
:104180006091AB0481E0611101C080E00C94F91EE4
:104190009091AF0481E0943009F080E06091AB042D
:1041A0000C94FE1E42E061EC81E00E94EF2342E2AB
:1041B00061EC84E00E94EF2342E261EC82E00E9425
:1041C000EF2342E260EC83E00E94EF239091AF0482
:1041D00081E0943009F080E06091AB040C94F01E13
:1041E0008091B104833009F462C030F48130D9F198
:1041F000823009F49EC008958A3009F48AC08B3059
:1042000009F470C0893009F051C08091B004813246
:1042100009F04CC08091B4049091B504009719F056
:10422000029709F043C08091E800877F8093E800FF
:104230008091E80082FF36C09091F3008091F200F7
:10424000029731F48091F100813011F0863021F431
:104250008091F100809397028091E8008B778093A2
:10426000E8000C9423248091B004813AF9F4809101
:10427000E800877F8093E8008091B4049091B504B2
:10428000892B61F460E287E792E070E00E943223BC
:104290008091E8008B778093E800089560E090E0DB
:1042A00080E0F3CF8091AF048111C2CF0895809157
:1042B000B004813AD9F78091B4049091B504892B68
:1042C000A9F78091E800877F8093E8008091E8005B
:1042D00080FFFCCF80911F018093F1008091E80066
:1042E0008E77BDCF8091B004813201F78091B40404
:1042F0009091B504892BD1F68091E800877F809357
:10430000E8000E9423248091B20480931F010C9442
:1043100070088091B004813249F68091E800877F6F
:104320008093E8000E9423248091B3048093980234
:1043300008958091B004813A09F0B8CF8091E800E7
:10434000877F8093E8008091E80080FFFCCF809118
:104350009802C2CF84B7877F84BF0FB6F894A89520
:1043600080916000886180936000109260000FBEB1
:1043700080E890E00FB6F89480936100909361001C
:104380000FBE0C94051F0E9473240E94D024E2EEFD
:10439000F0E080818460808378940C94592783E1D5
:1043A00091E00C94CC1D8091AF048530A9F48091EC
:1043B000AF04853011F00C94491F0E94081F8091B2
:1043C000AD048823A1F30E94351F882381F30E9446
:1043D0007E220E947008EBCF0895CF93DF93CDB774
:1043E000DEB7A0970FB6F894DEBF0FBECDBF8091A9
:1043F000AF04843009F583E08093E9008091E80000
:1044000082FF1AC08091E80090E085FF09C050E06B
:1044100040E060E270E0CE0101960E94E32291E06C
:104420008091E8008B778093E800992329F060E27F
:10443000CE0101960E94C315A0960FB6F894DEBF78
:104440000FBECDBFDF91CF9108950C942722292F65
:1044500033272330310521F168F42130310509F487
:1044600043C02230310509F444C090E080E030E0E0
:1044700020E026C02132310551F122323105A9F761
:104480006330710590F7FB01EE0FFF1FEA55FE4FF9
:10449000208131816D557E4FFB01808190E010C0FD
:1044A00099278130910581F0009729F00297E9F66C
:1044B000E0E1F4E002C0E0E5F4E0849190E09F01E7
:1044C000FA01318320830895E2E2F4E0F6CF63300D
:1044D000710558F6660F771FFB01E455FE4F2081EA
:1044E000318189E090E0ECCF82E190E02FEA34E086
:1044F000E7CF8BE590E024E534E0E2CF80E189BDB1
:1045000082E189BD09B400FEFDCF8091D8008F7D86
:104510008093D8008091E00082608093E0008091D9
:10452000E00081FDFCCF0895AF92BF92CF92DF9261
:10453000FF920F931F93CF93DF936C01EB018A01DE
:104540000E944224F82E811123C00115110539F073
:10455000F80180819181C81BD90BC80ED91EB12CDE
:10456000A12C2097A9F08091E80085FD22C08091C0
:10457000E8008E778093E80001151105A1F0F8019D
:1045800080819181A80EB91EB182A08285E0F82EAB
:104590008F2DDF91CF911F910F91FF90DF90CF90E2
:1045A000BF90AF9008950E9442248823D1F2F82E44
:1045B000EFCFF60181916F018093F1002197FFEF1A
:1045C000AF1ABF0ACECFAF92BF92CF92DF92FF92C7
:1045D0000F931F93CF93DF936C01EB018A010E942D
:1045E0004224F82E811123C00115110539F0F8017C
:1045F00080819181C81BD90BC80ED91EB12CA12C6A
:104600002097A9F08091E80085FD22C08091E80004
:104610008B778093E80001151105A1F0F8018081E6
:104620009181A80EB91EB182A08285E0F82E8F2D4F
:10463000DF91CF911F910F91FF90DF90CF90BF90AE
:10464000AF9008950E9442248823D1F2F82EEFCF34
:104650008091F100F60181936F012197FFEFAF1A6E
:10466000BF0ACECFFC018091B6049091B7048617A3
:104670009707A0F06115710529F49091E8009E77E5
:104680009093E80090E06115710551F4911108C014
:104690008091E80082FF34C080E00895BC01F2CF31
:1046A0008091AF048823C1F18530C1F18091E80089
:1046B00083FD30C08091E80082FDEACF8091E80060
:1046C00080FFE1CF8091F3002091F200382F611537
:1046D000710519F02830310558F091E02830310586
:1046E00009F090E02091E8002E772093E800CBCFEE
:1046F00081918093F100615071092F5F3F4FE7CFA7
:104700008091AF04882341F0853041F08091E8002A
:1047100083FFBECF81E0089582E0089583E008958D
:10472000FC018091B6049091B70486179707A0F01A
:104730006115710529F48091E8008E778093E80077
:1047400090E06115710551F4911108C08091E80065
:1047500082FF35C080E00895BC01F2CF8091AF04A4
:104760008823C9F18530C9F18091E80083FD31C00B
:104770008091E80082FDEACF8091E80080FFE1CFE0
:104780008091F3002091F200382F6115710519F026
:104790002830310558F091E02830310509F090E0DB
:1047A0008091E8008E778093E800CBCF849180934E
:1047B000F1003196615071092F5F3F4FE6CF809134
:1047C000AF04882341F0853041F08091E80083FFF9
:1047D000BDCF81E0089582E0089583E00895982F89
:1047E000973028F08F708093E90081E008959093CE
:1047F000E900242F762F50E0981731F07091EC00EB
:104800002091ED005091F00021FD02C09F5FE8CFA4
:104810003091EB003E7F3093EB003091ED003D7F17
:104820003093ED003091EB0031603093EB007093EA
:10483000EC002093ED005093F0002091EE0027FD56
:10484000E5CF80E008958091B00487FF13C0809188
:10485000E80082FF06C08091E8008B778093E80033
:1048600004C08091AF048111F2CF08958091AF040C
:104870008823D9F38091E80080FFF8CF8091E80089
:104880008E77ECCF2091E4003091E50095E6A90108
:104890002091EC00822F817020FF06C08091E800FB
:1048A00080FF06C080E008952091E80022FD1AC034
:1048B0008091AF04882389F0853089F08091EB00E6
:1048C00085FD0FC02091E4003091E50042175307A9
:1048D000F9F29150E1F684E0089582E0089583E0D2
:1048E000089581E008950E94E1240E94E924E0EE09
:1048F000F0E0808181608083E8EDF0E080818F7757
:10490000808319BCA7EDB0E08C918E7F8C93808161
:104910008F7E80831092AE0408950F931F93CF93E0
:10492000DF930E94E1240E94E924C8EDD0E0888151
:104930008F77888388818068888388818F7D88834A
:1049400019BC1092AF041092AB041092AD041092F7
:10495000AC0400EE10E0F80180818B7F80838881B9
:104960008160888342E060E080E00E94EF23E1EE16
:10497000F0E080818E7F8083E2EEF0E080818160D4
:104980008083808188608083F80180818E7F80832E
:10499000888180618883DF91CF911F910F91089565
:1049A000E8EDF0E080818F7E8083E7EDF0E08081AC
:1049B0008160808384E082BF81E08093AE040C94A8
:1049C0008D24E8EDF0E080818E7F80831092E200FC
:1049D00008951092DA001092E10008951F920F924C
:1049E0000FB60F9211242F933F934F935F936F93C2
:1049F0007F938F939F93AF93BF93EF93FF93809198
:104A0000E10082FF0BC08091E20082FF07C080912D
:104A1000E1008B7F8093E1000E9458278091DA00AB
:104A200080FF19C08091D80080FF15C08091DA0006
:104A30008E7F8093DA008091D90080FF96C080E15C
:104A400089BD82E189BD09B400FEFDCF81E080937C
:104A5000AF040E94AD208091E10080FF19C08091D9
:104A6000E20080FF15C08091E2008E7F8093E2001B
:104A70008091E20080618093E2008091D8008062A2
:104A80008093D80019BC85E08093AF040E94C020B9
:104A90008091E10084FF2BC08091E20084FF27C059
:104AA00080E189BD82E189BD89B5982F917080FF31
:104AB000FBCF8091D8008F7D8093D8008091E1005A
:104AC0008F7E8093E1008091E2008F7E8093E200F0
:104AD0008091E20081608093E2008091AB048823A2
:104AE00009F449C084E08093AF040E94C8208091FB
:104AF000E10083FF29C08091E20083FF25C08091FF
:104B0000E100877F8093E10082E08093AF04109200
:104B1000AB048091E1008E7F8093E1008091E20000
:104B20008E7F8093E2008091E20080618093E200BA
:104B300042E060E080E00E94EF238091F000886016
:104B40008093F0000E94BE20FF91EF91BF91AF9142
:104B50009F918F917F916F915F914F913F912F9195
:104B60000F900FBE0F901F90189519BC1092AF04B4
:104B70000E94BB2070CF8091E30087FD93E090936B
:104B8000AF04B3CF1F920F920FB60F9211242F9341
:104B90003F934F935F936F937F938F939F93AF93C5
:104BA000BF93CF93DF93EF93FF93D091E900DF7032
:104BB0008091EC00C82FC17080FDC0E81092E90020
:104BC0008091F000877F8093F00078940E94062601
:104BD0001092E9008091F00088608093F000CD2B66
:104BE000CF70C093E900FF91EF91DF91CF91BF911A
:104BF000AF919F918F917F916F915F914F913F9175
:104C00002F910F900FBE0F901F9018951F93CF9369
:104C1000DF93CDB7DEB7AA970FB6F894DEBF0FBE0D
:104C2000CDBF80EB94E02091F100FC012193CF01F6
:104C3000F4E0883B9F07B9F70E94F0208091E800DC
:104C400083FF1EC18091B0049091B1049A3008F0A6
:104C500017C1E92FF0E0E95DF74D0C949C278038EF
:104C600099F0823809F00CC18091B4048F708730BC
:104C700008F006C18093E9008091EB0085FB88274E
:104C800080F91092E90006C08091AC049091AD04C7
:104C9000911182609091E800977F9093E800809353
:104CA000F1001092F1008091E8008E77E5C0882332
:104CB00009F4D3C0823009F0E3C08091B2048111BD
:104CC000D6C08091B4048F702FEF280F263008F0E3
:104CD000D7C08093E9002091EB0020FFC8C093303B
:104CE00031F48091EB0080628093EB00C0C0909122
:104CF000EB0090619093EB0021E030E001C0220FC7
:104D00008A95EAF72093EA001092EA008091EB007E
:104D10008860EACF8111B4C01091B2041F778091EE
:104D2000E3008078812B8093E3008091E800877F07
:104D30008093E8000E9423248091E80080FFFCCF4C
:104D40008091E30080688093E30082E0111183E0AA
:104D50008093AF0495C08058823008F091C0809154
:104D6000B2049091B3048C3D23E09207A1F583E057
:104D70008A838AE289834FB7F894DE01139620E094
:104D80003EE051E2E32FF0E050935700E49120FF22
:104D900003C0E295EF703F5FEF708E2F90E0EA3036
:104DA000C0F0C7968D939D932F5F243159F74FBF65
:104DB0008091E800877F8093E8006AE270E0CE018E
:104DC00001960E9432238091E8008B778093E8005F
:104DD00057C0C096E7CF6091B4047091B504AE019E
:104DE0004F5F5F4F0E942522BC01892B09F448C008
:104DF0009091E800977F9093E80089819A810E94C2
:104E00009023E1CF8038E1F58091E800877F80939F
:104E1000E8008091AB048093F10045CF811130C050
:104E20009091B204923060F58091E800877F809382
:104E3000E8009093AB040E9423248091AB04882364
:104E400011F084E005C08091E30087FDFACF81E096
:104E50008093AF040E94D22013C08091B2048130AD
:104E600079F481E0933009F080E08093AD041092F2
:104E7000E9008091E800877F8093E8000E94232466
:104E80008091E80083FF0AC08091E800877F8093CB
:104E9000E8008091EB0080628093EB00AA960FB649
:104EA000F894DEBF0FBECDBFDF91CF911F91089563
:104EB0000895CF938091AF048823A1F0C091E900B9
:104EC000CF709091EC00892F817090FD80E8C82B05
:104ED0001092E9008091E80083FD0E940626CF70C1
:104EE000C093E900CF910895AA1BBB1B51E107C0F5
:104EF000AA1FBB1FA617B70710F0A61BB70B881F6A
:104F0000991F5A95A9F780959095BC01CD010895F8
:104F100097FB072E16F4009407D077FD09D00E9466
:104F2000742707FC05D03EF4909581959F4F089516
:104F3000709561957F4F0895EE0FFF1F0590F491D6
:104F4000E02D0994692796276927782787277827EE
:104F50000895FB01DC0104C08D910190801921F4BA
:104F600041505040C8F7881B990B0895F999FECF1E
:104F700092BD81BDF89A992780B50895A8E1B0E067
:104F800042E050E00C94EA27262FF999FECF92BD1B
:104F900081BDF89A019700B4021639F01FBA20BDFE
:104FA0000FB6F894FA9AF99A0FBE08950396272F30
:104FB0000E94C5270E94C427252F0E94C527242FA1
:104FC0000C94C5270196272F0E94C5270C94C4274F
:104FD000DC01CB01FC01F999FECF06C0F2BDE1BDB9
:104FE000F89A319600B40D9241505040B8F70895A8
:104FF000F894FFCF54065406850685061807340733
:10500000B406B4063F07A607B507B5077F087F08B3
:10501000880888088A088808880888087F087F0820
:105020008F08880888088F08D215DC1501160D1620
:10503000181623162616261626162616261629169E
:105040002D16351642164F165216551662162F2675
:1050500057264027572640278A26AB264027022777
:025060000E2719
:10506200C800FA012808641E140A321E0021007FBB
:10507200220003EC1F1120F01F7F207B20EF1F0175
:10508200E200E900EA00B500B600B700CD008301F6
:10509200CC008A01920194012102230224022502FA
:1050A200260227022A02B300B4006F007000818238
:1050B20083E200E900EA00B500B600B700CD008344
:1050C20001CC008A019201940121022302240225CB
:1050D20002260227022A02B300B4006F0070008188
:1050E2008283F0F1F4F5F637C6F767000810181856
:1050F20010080000FF0100010000FFFF0000010096
:1051020001FF004022B69905C104E30466047F044E
:025112009F04F8
:00000001FF
